:100000000C94E3050C9495280C94C2280C940B06D0
:100010000C940B060C940B060C940B060C940B061C
:100020000C940B060C940B060C94A10C0C940B0670
:100030000C940B060C940B060C940B060C940B06FC
:100040000C94EF280C940B060C94972C0C94D22C47
:100050000C940B060C940B060C940B060C940B06DC
:100060000C940B060C940B060D1C141C141C0D1C7C
:10007000141C141C141C141C141C141C141C141C00
:10008000141C141C141C141C141C7C1B141C141C89
:10009000141C141C141CDF1A141C141C141C141C17
:1000A000141C141C141C141C141C141C141C141CD0
:1000B000141C141C141C881B881B881B881B881B81
:1000C000881B881B881B881B141C141C141C141CE4
:1000D000141C141CE41A871B871B871B871B141C0A
:1000E0009E1BA61BAE1BB61BBE1BC61BCE1BD61B68
:1000F000E01BEA1BF41BFE1B2B1BEB1A141C141C2D
:10010000141C141C7C1B141C141C141C141C141C08
:10011000141C141C141C861B861B861B861B141C9B
:100120009E1BA61BAE1BB61BBE1BC61BCE1BD61B27
:10013000E01BEA1BF41BFE1B2B1BEB1A141C141CEC
:10014000141C141C7C1B456E746572206D656E75E5
:100150002E2E2E00546F67676C6564206D69637284
:100160006F50504D00546F67676C656420696E7600
:1001700065727465642050504D2100546F67676C40
:100180006564205458206D7574696E672100546F42
:1001900067676C65642074656C656D657472792140
:1001A0000050726F746F636F6C206572726F722093
:1001B000776974682052580054696D656F757420B2
:1001C0007768656E20636F6E6E656374696E672015
:1001D000746F20525800507265737320616E7920DD
:1001E0006B657920746F2063616E63656C00436F8B
:1001F0006E6E656374696E6720746F2052582C2090
:10020000706F776572207570207468652052582071
:1002100028776974682062696E6420706C75672045
:100220006966206E6F74207573696E6720616C77E4
:100230006179732062696E642900546F67676C6529
:10024000642027696D6D656469617465206F7574DC
:100250007075742700546F67676C65642027736C32
:10026000617665206D6F64652700546F67676C6504
:10027000642027616C776179732062696E6427005E
:10028000546F67676C65642050504D206368616EE1
:100290006E656C206C696D697400536574205253EF
:1002A000534920696E6A656374696F6E2063686183
:1002B0006E6E656C2028303D3D64697361626C65CB
:1002C00029005365742050504D206D696E696D751D
:1002D0006D2073796E630053657420626561636F8E
:1002E0006E20696E74657276616C0053657420626D
:1002F0006561636F6E2064656C617900536574207D
:10030000626561636F6E206672657175656E637993
:1003100020696E20487A3A20303D64697361626CCE
:10032000652C2050783D504D52206368616E6E659B
:100330006C20782C2046783D465253206368616ECD
:100340006E656C2078005365742050574D2073748F
:100350006F702064656C6179202830206469736156
:10036000626C65642C20312D323535203D3D2030C6
:100370002E3173202D2035306D696E290053657440
:100380002050504D2073746F702064656C6179202B
:1003900028302064697361626C65642C20312D32D1
:1003A0003535203D3D20302E3173202D2035306DE8
:1003B000696E2900536574206661696C73616665B6
:1003C0002064656C61792028302064697361626CF7
:1003D00065642C20312D323535203D3D20302E31C5
:1003E00073202D2035306D696E29002A2A2A2A2A89
:1003F0002A2A2A2A2A2A2A2A2A2A2A2A2A2A2A2A5D
:100400002A2A2A2A2A2A2A2A0052582041636B655E
:1004100064202D2072657665727420737563636540
:10042000737366756C21002A2A2A2A2A2A2A2A2A04
:100430002A2A2A2A2A2A2A2A2A2A2A2A2A2A2A2A1C
:100440002A2A2A2A002A2A2A2A2A2A2A2A2A2A2A36
:100450002A2A2A2A2A2A2A2A2A2A2A2A2A2A2A2AFC
:100460002A2A0052582041636B6564202D20757044
:1004700064617465207375636365737366756C215D
:10048000002A2A2A2A2A2A2A2A2A2A2A2A2A2A2AF6
:100490002A2A2A2A2A2A2A2A2A2A2A2A2A2A0056BA
:1004A000616C69642063686F69636573206172655C
:1004B0003A205B315D2D5B31365D20286368616ECB
:1004C0006E656C20312D31362900536574206F75AF
:1004D0007470757420666F7220706F727420005B88
:1004E000585D2061626F7274206368616E67657326
:1004F00020616E64206578697420525820636F6EA5
:10050000666967005B535D2073617665207365746F
:1005100074696E677320746F205258005B525D20BF
:100520007265766572742052582073657474696EB2
:10053000677320746F2064656661756C7473005511
:100540007365206E756D62657273205B312D445D3D
:1005500020746F206564697420706F727473205BFF
:10056000452D515D20666F722073657474696E67E6
:100570007300202D20726563656976657220636F54
:100580006E666967757261746F722C207278207361
:100590007720000A0A6F70656E4C52536E67200018
:1005A0005365742073657269616C20626175647251
:1005B0006174653A200056616C69642063686F69F4
:1005C0006365733A2031202D20342B34202F2032C4
:1005D000202D2038202F2033202D20382B34202F81
:1005E0002034202D203132202F2035202D20313273
:1005F0002B34202F2036202D2031360053657420D7
:100600004368616E6E656C20636F6E6669673A2041
:1006100000536574204461746172617465202830F0
:100620002D32293A200053657420486F702063688A
:10063000616E6E656C7320286D61782032342C20D9
:1006400073657061726174656420627920636F6D97
:100650006D6173292076616C69642076616C7565C3
:100660007320312D3235353A20005365742063688C
:10067000616E6E656C2073706163696E67202878A7
:1006800031306B487A293A20005365742052462055
:10069000706F7765722028302D37293A2000536516
:1006A00074205246206D6167696320286865782947
:1006B00020652E672E203078444541444630304432
:1006C0003A2000536574206261736520667265711B
:1006D00075656E63792028696E20487A293A200072
:1006E0005B5A5D20656E746572207265636569761C
:1006F000657220636F6E66696775726174696F6E8B
:10070000207574696C79005B465D20646973706C58
:1007100061792061637475616C20667265717565BD
:100720006E636965732075736564005B525D206359
:10073000616C63756C6174652072616E646F6D20AD
:100740006B657920616E6420686F70206C697374CA
:10075000005B495D207265696E697469616C697AD4
:10076000652073657474696E677320746F20736B92
:10077000657463682064656661756C7473005B58AA
:100780005D20726576657274206368616E6765735B
:1007900020616E642065786974206D656E75005BFC
:1007A000535D20736176652073657474696E677339
:1007B00020746F20454550524F4D20616E64206576
:1007C000786974206D656E7500557365206E756D62
:1007D00062657273205B302D395D20746F20656413
:1007E000697420706172616D657465727300202D8B
:1007F0002053797374656D20636F6E6669677572D7
:100800006174696F6E000A0A6F70656E4C52536EA8
:100810006720005129204F757470757420626566D9
:100820006F7265206C696E6B20283D465329203A13
:100830002000502920536C617665206D6F6465201F
:10084000286578706572696D656E74616C293A20EF
:10085000004F292054696D65642042494E4420614F
:1008600074207374617274757020203A20004E29D0
:100870002050504D206F7574707574206C696D69CF
:1008800074656420202020203A20004449534142CE
:100890004C4544004D292050504D2052535349207F
:1008A000746F206368616E6E656C202020203A2092
:1008B000004C292050504D206D696E696D756D207A
:1008C00073796E63202875732920203A20004449EB
:1008D0005341424C4544004B29204661696C736189
:1008E000666520626561636F6E20696E74762E2086
:1008F00028312D32353573293A20004A29204661A6
:10090000696C7361666520626561636F6E20646502
:100910006C61792028302D323535203D3E20313034
:1009200073202D203135306D696E293A2000492918
:10093000204661696C7361666520626561636F6EF4
:10094000206672712E203A200048292050574D20F1
:1009500073746F702064656C6179202020202020E2
:10096000203A200047292050504D2073746F70208A
:1009700064656C6179202020202020203A200046E8
:1009800029204661696C736166652064656C6179D4
:10099000202020202020203A200050574D2063683E
:1009A000616E6E656C200066756E6374696F6E3A79
:1009B00020002920706F727420004454462055484E
:1009C000462033322D6269742031306368004F70E5
:1009D000656E4C52536E675258206D696E692034B3
:1009E0002F36636800466C7974726F6E2F4F726198
:1009F0006E67655258205548462038636800525843
:100A000020747970653A200044697361626C656492
:100A100000487A00203D3D200043616C63756C61A5
:100A2000746564207061636B657420696E746572AF
:100A300076616C3A20004229204D6963726F20284C
:100A400068616C66292050504D202020203A0041DA
:100A50002920496E7665727465642050504D206976
:100A60006E20202020203A003029204D757465200A
:100A700062757A7A657220286D6F73746C79293A81
:100A80000039292053657269616C20626175647256
:100A90006174653A00736D617274506F72740046D0
:100AA00072536B79005472616E73706172656E740B
:100AB0000044697361626C65640038292054656C78
:100AC000656D657472793A2020202020202000373F
:100AD00029204368616E6E656C20636F6E6669677E
:100AE0003A202000362920446174617261746520C7
:100AF00028302D32293A20202000352920486F70D7
:100B0000206368616E6E656C733A2020202020009F
:100B10003429204368616E6E656C2073706163696F
:100B20006E673A202000332920524620706F776587
:100B3000722028302D37293A2020200032292052D7
:100B400046206D616769633A202020202020202004
:100B500020003129204261736520667265717565D8
:100B60006E63793A20202000000000002400270056
:100B70002A0000000000250028002B0000000000D3
:100B800023002600290004040404040404040202CF
:100B900002020202030303030303010204081020FC
:100BA0004080010204081020010204081020000007
:100BB000000700020100000304060000000000001E
:100BC0000000390F8B2E11241FBECFEFD8E0DEBFFF
:100BD000CDBF13E0A0E0B1E0E8E5FFE502C005907D
:100BE0000D92AA3FB107D9F716E0AAEFB3E001C012
:100BF0001D92A33AB107E1F71BE0C6ECDBE004C0AD
:100C00002297FE010E94642FC23CD107C9F70E94BF
:100C1000D02E0C94AA2F0C940000A0E0B0E0E3E1E9
:100C2000F6E00C947B2FEC01A880B980CA80DB80B1
:100C3000A114B104C104D10441F484E2A82E89EDC9
:100C4000B82E8BE5C82E87E0D82EC601B5012DE160
:100C500033EF41E050E00E94332F27EA31E440E0D7
:100C600050E00E94DF2E7B018C01C601B5012DE111
:100C700033EF41E050E00E94332FCA01B9012CEE5E
:100C800034EF4FEF5FEF0E94DF2E6E0D7F1D801F50
:100C9000911F97FF04C06150704080409048688366
:100CA00079838A839B839B01AC015F77B901CA0179
:100CB000CDB7DEB7EAE00C94972F0E940D06089599
:100CC00084E193E00E940D060895609314037093ED
:100CD000150380931603909317030895A0E0B0E0E6
:100CE000E4E7F6E00C94742FEC012B016A01611526
:100CF000710519F0FB0191838083C114D10449F07F
:100D0000C6010297839728F020E030E040E050E0F1
:100D1000DCC0A9908A2D90E00E94682F892BC9F72A
:100D2000FDE2AF1621F4A9903324339405C08BE281
:100D3000A81609F4A9903324C114D10421F0E0E1EC
:100D4000CE16D10411F5F0E3AF1669F48881883727
:100D500011F0883541F4A980229682E0382A20E1FA
:100D6000C22ED12C12C0C114D10479F4E0E3AE1626
:100D700059F199E9E92E99E9F92E99E9092F99E1B3
:100D8000192F8AE0C82ED12C3AC0FAE0CF16D10430
:100D900091F080E1C816D10429F0E8E0CE16D10424
:100DA000F9F415C0BFEFEB2EBFEFFB2EBFEF0B2FFB
:100DB000BFE01B2F24C0A9E9EA2EA9E9FA2EA9E970
:100DC0000A2FA9E11A2F1BC0F8E0CF2ED12CEFEF8C
:100DD000EE2EEFEFFE2EEFEF0E2FEFE11E2F0FC0E6
:100DE0009601442737FD4095542F6FEF7FEF8FEF2B
:100DF0009FEF0E94112FC901DA017C018D0120E0D3
:100E000030E040E050E060E03601882477FC8094D8
:100E1000982C70EDB72EBA0CF9E0FB1570F48A2D02
:100E200081548A3118F499ECB92E06C08A2D815666
:100E30008A3148F589EAB82EBA0C8B2D90E08C15D2
:100E40009D050CF56F3FE9F0E216F3060407150760
:100E5000B8F0CA01B901A40193010E94DF2E9B01E1
:100E6000AC018B2D90E0A0E0B0E0280F391F4A1FA5
:100E70005B1F281739074A075B0710F061E001C0C4
:100E80006FEFA990C6CF4114510451F0662311F0C1
:100E9000219703C031FE04C02297F201D183C083A1
:100EA00030FE07C050954095309521953F4F4F4FEC
:100EB0005F4F67FF0AC082E290E09093A2068093A2
:100EC000A1062FEF3FEF4FEF5FEFB901CA01CDB79A
:100ED000DEB7E1E10C94902FFC0188279927E89474
:100EE00021912032E9F3293010F02E30C8F32B3253
:100EF00041F02D3239F4689404C00E94C107820F7A
:100F0000911D219120532A30C0F31EF490958195B4
:100F10009F4F08954AEF53E00E948F07089500976E
:100F200031F4DA018D919C91009709F40EC0DC0137
:100F3000FB013D912191222319F03217C9F3FACF19
:100F4000332331F4DA011D921C92882799270895E2
:100F50001197AF93BF93FB013D912191321771F42B
:100F6000332321F488279927119702C01E921196E6
:100F7000FA01A193B0839F918F910895222369F77D
:100F8000EACF7AE0979F902D879F802D910D1124B5
:100F900008958091FC03813019F482E08093FC0372
:100FA0008091FC03833019F484E08093FC0308955E
:100FB000009721F19C0140E050E068E478EE81E088
:100FC00090E00E94332FC901DA018F3F9105A105FE
:100FD000B10531F028F08FEF90E0A0E0B0E008C05C
:100FE0000097A105B10521F481E090E0A0E0B0E018
:100FF0008093B3008091B000806103C08091B00005
:101000008F7E8093B000089580912604E82FF0E051
:101010003496DF0126E0AA0FBB1F2A95E1F720E0F6
:1010200030E040E050E060E070E0F999FECFCB01A5
:101030008A0F9B1F92BD81BDF89A80B5542F432F14
:10104000322F2227280F311D411D511D6F5F7F4F09
:101050006430710551F72E513E4B414C5E4D19F0F5
:1010600020E030E01FC09F0186E0220F331F8A95E9
:10107000E1F72C5F3F4FEDEFF3E0F999FECF32BD82
:1010800021BDF89A80B581932F5F3F4F84E0E6320F
:10109000F80799F720E030E08091FD03893011F4E2
:1010A00021E030E0C901089589E08093FD0380E0EC
:1010B00092ECA1E0B0E08093FE039093FF03A09335
:1010C0000004B093010487E080930A0480EC92E965
:1010D000ADEEB9E18093020490930304A09304045D
:1010E000B093050485E080930B048DEE9EEFADEA8E
:1010F000BEED8093060490930704A0930804B09378
:101100000904ACE0B4E080E090E0863010F0E0E06C
:1011100004C0FC01ED51FC4FE081ED930196883154
:10112000910599F782E0809324048AE08093250456
:1011300008958436910520F4BC0180E090E025C03C
:101140008E3B910550F48A559040BC0180E090E0C0
:101150002AE030E040E050E016C0823D910550F4B6
:10116000845B9040BC0180E090E024E630E040E009
:1011700050E009C08D5C9040BC0180E090E028E523
:1011800032E040E050E00E94DF2E24E630E040E014
:1011900050E00E94DF2E089590E08C599F4F0E94EE
:1011A00099080895DC019896EC91F0E0E770F070F2
:1011B000E552FC4F808108958F929F92AF92BF922B
:1011C000CF92DF92EF92FF920F931F938C010E94B8
:1011D000D208D80197962C9130E043E150E0249F4B
:1011E000F001259FF00D349FF00D1124E85EFC4FB7
:1011F00080809180A280B38090E00F96AA2797FD0F
:10120000A095BA2FBC01CD0120E43FE14DE750E0AD
:101210000E94DF2EA50194010E94112F69017A011D
:1012200080ED97E0A0E0B0E0C80ED91EEA1EFB1EDC
:10123000D80198968C91887181F060E07EEE8AEBFF
:101240009BE0A50194010E94112F28513C4F4F4F64
:101250005F4FC20ED31EE41EF51E87EE93E0A0E0A2
:10126000B0E0C80ED91EEA1EFB1EC701B60128EE6B
:1012700033E040E050E00E94112FCA01B90128EE8E
:1012800033E040E050E00E94DF2E1F910F91FF906D
:10129000EF90DF90CF90BF90AF909F908F90089588
:1012A0008F3F910509F010F480E0089522E080302E
:1012B000920710F481E008958050934010F083E08D
:1012C000089582E00895CF92DF92FF920F931F93CB
:1012D000CF93DF93F82FEB016A01182F1695E0E00A
:1012E00088819981D6018C938A819B8111968C93F8
:1012F00011978C819D8112968C9312978E819F817C
:1013000013968C931397288139814A815B816C8174
:101310007D818E819F819295990F990F907C832F6B
:101320008370982B852F8370880F880F982B872FB9
:1013300083708295807F982B14969C9385E090E033
:10134000C80ED91E2896EF5F1E1750F6F0FF21C079
:10135000888199810E945009F82E8A819B810E9480
:101360005009182F8C819D810E945009082F8E8171
:101370009F810E945009F294FF0CFF0C50ECF52263
:101380001295107F1F29182B000F000F012BD6017B
:101390000C93DF91CF911F910F91FF90DF90CF9031
:1013A000089523E08032920718F420E030E026C050
:1013B00023E0883E920748F49C012F513340F4E02B
:1013C00036952795FA95E1F719C027E0803D9207F9
:1013D00020F49C012C5D334011C028E0883992072D
:1013E00018F02FEF33E00AC09C01285C3740E4E09E
:1013F00036952795EA95E1F72D503C4FC9010895A0
:101400009C013695279525753575821B930B9C019C
:101410003695279536952795237333738373937386
:10142000280F391FC90144E0969587954A95E1F741
:10143000820F931F8F709F7021E031E0AC01429FBB
:10144000C001439F900D529F900D1124892F089544
:10145000382F20E08091E8059091E90582279327B5
:1014600040E061E270E19C01220F331F97FF04C04E
:10147000C9018627972701C0C9014F5F483099F7F6
:101480009093E9058093E8050895882339F02D9815
:1014900000002B9A00002D9A000008952D9800005E
:1014A0002B9800002D9A000008952D9A000083B11A
:1014B0002D98000090E0F4E096958795FA95E1F775
:1014C000817008950F931F93082F5C9A2D985C9854
:1014D00010E0802F80780E94450A000F1F5F1830AF
:1014E000C1F72D981F910F9108958F770E94620A7E
:1014F00008950F931F93082F10E0802F80780E948B
:10150000450A000F1F5F1830C1F72D981F910F91EA
:1015100008950F931F932D9880E000E0182F110F6E
:101520000E94550A810F0F5F0830C1F71F910F917C
:1015300008950E94750A0E94890A5C9A08951F9373
:10154000162F80680E94620A812F0E94790A5C9A95
:101550001F9108951F93109106041827EDEFF3E0F3
:10156000E80FF11D89E767850E949F0A8DE3612FCF
:101570000E949F0A82E4612F0E949F0A1F91089592
:1015800086E20E94990A08950F931F938C018CE1C3
:10159000F80164810E949F0A8DE1F80165810E9433
:1015A0009F0A8EE1F80166810E949F0A80E2F8019D
:1015B00067810E949F0A81E2F80160850E949F0A6C
:1015C00082E2F80161850E949F0A83E2F801628548
:1015D0000E949F0A84E2F80163850E949F0A85E2C7
:1015E000F80164850E949F0A8AE2F80165850E94DD
:1015F0009F0A8EE6F80166850E949F0A8FE6F80131
:1016000067850E949F0A80E7F80160890E949F0A0F
:1016100081E7F80161890E949F0A82E7F8016289E7
:101620000E949F0A1F910F910895EF92FF920F93CE
:101630001F93CF93DF937B018C01603028E3720707
:101640002CE982072CE1920728F520E836E948E9E1
:1016500050E00E94112FE9016897B90180E090E005
:1016600020E839E647E65FEF0E94DF2E6E0D7F1D12
:10167000801F911F02E0660F771F881F991F0A9530
:10168000D1F721E732E040E050E00E94112F8901BC
:1016900080E421C020E03DE241E351E00E94112FAF
:1016A000E9016897B90180E090E020E033ED4EEC6D
:1016B0005EEF0E94DF2E6E0D7F1D801F911F660F53
:1016C000771F881F991F21E732E040E050E00E9419
:1016D000112F890180E69E012F71622F680F85E727
:1016E0000E949F0A86E7612F0E949F0A87E7602F6A
:1016F0000E949F0ADF91CF911F910F91FF90EF9071
:1017000008959F92AF92BF92CF92DF920F93DF9393
:10171000CF9300D000D0CDB7DEB7982E83E00E94E3
:10172000990A8093420484E00E94990A80934304BA
:1017300086E060E00E949F0A87E061E00E949F0AC5
:1017400089E06FE70E949F0A8AE065E00E949F0A95
:101750008BE065E10E949F0A8CE062E10E949F0A93
:101760008DE06DEF0E949F0A8EE060E00E949F0A6C
:10177000992019F087E793E008C08091240423E1C1
:10178000829FC0011124885E9C4F0E94C40A80E39E
:101790006CE80E949F0A82E36FE00E949F0A83E345
:1017A00062E40E949F0A84E36AE00E949F0A85E344
:1017B0006AE20E949F0A86E36DE20E949F0A87E325
:1017C00064ED0E949F0A88E360E00E949F0A89E31B
:1017D00060E00E949F0A992049F02EE1A22E2EEB94
:1017E000B22E21ECC22E2EEDD22E08C0A0900604FF
:1017F000B0900704C0900804D09009040AE38D2D2E
:101800009927AA27BB2789839A83AB83BC83802F20
:1018100069810E949F0A802F8B5F69810E949F0AC5
:10182000DC2CCB2CBA2CAA240F5F0E3341F783E4B7
:101830006FEF0E949F0A84E46FEF0E949F0A85E485
:101840006FEF0E949F0A86E46FEF0E949F0A992023
:1018500019F08DE666E003C08DE660910A040E94EF
:101860009F0A89E760E00E949F0A8AE760910B0463
:101870000E949F0A83E760E00E949F0A84E760E07D
:101880000E949F0A992029F060EC72E98DEE99E19F
:1018900008C0609102047091030480910404909147
:1018A00005040E94150B0F900F900F900F90CF9191
:1018B000DF910F91DF90CF90BF90AF909F900895F0
:1018C00087E061E00E949F0A8EE764E20E949F0A1F
:1018D00088E063E00E949F0A88E060E00E949F0A1F
:1018E00087E065E00E949F0A85E062E00E949F0A0F
:1018F00083E00E94990A8093420484E00E94990A3E
:10190000809343040895582F40915305842F90E00D
:10191000FC01EF70F0709F012F5F3F4F64E09595E1
:1019200087956A95E1F72817390751F0ED5BFA4F73
:101930005083842F8F5F8F70407F842B809353055B
:1019400008951F920F920FB60F9211241F932F9399
:101950003F934F935F936F937F938F939F93AF9337
:10196000BF93CF93DF93EF93FF93C0918600D09105
:101970008700209195053091960580917405882304
:1019800009F047C0CE01821B930B9C018091250476
:1019900087FD02C03695279599E0253C390708F167
:1019A0008091AA038630D0F08091AA038F3FB1F0D6
:1019B00020E00EC0E22FF0E0EE0FFF1FDF01AB587A
:1019C000BA4F8D919C91E657FC4F918380832F5F96
:1019D0008091AA03281770F3109273051092AA033E
:1019E00018C082E02D3B380760F18091AA03803156
:1019F00040F51091AA03C9010E94D109E12FF0E03E
:101A0000EE0FFF1FEB58FA4F918380831F5F1093F7
:101A1000AA03D0939605C0939505FF91EF91DF91AE
:101A2000CF91BF91AF919F918F917F916F915F9176
:101A30004F913F912F911F910F900FBE0F901F90CC
:101A400018958FEF8093AA03E4CF83E08093800002
:101A50008AE9809381008091250486FD05C08091EC
:101A600081008064809381008FEF9FEF90938900C5
:101A70008093880080916F00806280936F0008954A
:101A80006F3020F086958695805408958DE0689F8C
:101A9000802D11240895982F8091E105882329F441
:101AA000933009F043C081E005C0813049F49130A2
:101AB00021F482E08093E10508951092E1050895F4
:101AC000803190F5E82FF0E0EB58FA4F90838F5F6C
:101AD0008093E105803151F520917405A7E7B5E0C9
:101AE000213039F41196EC911197E695E6958C9199
:101AF00009C08D919C911197E92FE695E695E695A1
:101B000096958795E03140F4F0E090E0EE0FFF1FEE
:101B1000E657FC4F9183808310927305129685E0FF
:101B2000A538B807E9F608951092E10508950F93D6
:101B30001F93CF93DF939091E105992339F48F3070
:101B400009F002C181E08093E105FEC0983148F4BC
:101B5000E92FF0E0EC58FA4F80839F5F9093E10506
:101B6000F3C0983109F0EEC0882309F0EBC0C0E063
:101B7000D0E00BE010E0DE0163E0AA0FBB1F6A9526
:101B8000E1F7C09FB001C19F700DD09F700D11246F
:101B9000FB01EB58FA4F80812181922F9770959528
:101BA0008795FD01EE0FFF1FE657FC4F9183808361
:101BB000FB01EA58FA4F30813695369536952181EA
:101BC000422F4295440F407E842F832B26952695E5
:101BD0002695922F977095958795FD01EE0FFF1F23
:101BE000E457FC4F91838083FB01E958FA4F8081D1
:101BF00082958695869583704181942F990F990FD0
:101C0000292F282B429546954695437082818170F5
:101C1000880F880F382F342B35952795FD01EE0F4F
:101C2000FF1FE257FC4F31832083FB01E758FA4F37
:101C3000308136952181422F479544274795842F3F
:101C4000832B2695922F977095958795FD01EE0F22
:101C5000FF1FE057FC4F91838083FB01E658FA4F4A
:101C6000308132953F702181422F4295407F842FF1
:101C7000832B22952F70922F977095958795FD0154
:101C8000EE0FFF1FEE56FC4F91838083FB01E5585A
:101C9000FA4F8081881F8827881F4181942F990FD0
:101CA000292F282B441F4427441F82818370880FCB
:101CB000382F342B35952795FD01EE0FFF1FEC567D
:101CC000FC4F31832083FB01E358FA4F3081369576
:101CD00036952181422F4295440F440F407C842F3A
:101CE000832B26952695922F977095958795AA0F09
:101CF000BB1FFD01EA56FC4F9183808362587A4FE7
:101D0000FB0120812295269527704181342F330FC6
:101D1000330F330F832F822B942F929596959770C4
:101D200095958795A856BC4F11969C938E932196B6
:101D3000C230D10509F01FCF80918B0583FD02C011
:101D4000109273051092E105DF91CF911F910F91D1
:101D50000895DF92EF92FF920F931F93CF93DF933B
:101D6000682F4091E105442359F4883AB1F4109268
:101D7000E9051092E80588EA0E94280A81E06FC010
:101D8000413019F48093E60504C0423031F4809369
:101D9000E705862F0E94280A5DC07091E705272F6E
:101DA00030E0220F331FE42FF0E0C90102968E17B6
:101DB0009F0734F0433268F7EE58FA4F6083E9CF5B
:101DC0002D5F3F4F4091E8055091E905E217F30779
:101DD00049F4962F80E0482759275093E90540930E
:101DE000E80538C0862F90E04817590789F580919B
:101DF000E605813069F5713118F080E18093E705DF
:101E0000D090E705F5E7EF2EF5E0FF2E00E010E0BB
:101E10001BC0F701D081C0E0818190E08C2B9D2B0D
:101E2000E3E096958795EA95E1F70E94D109F801DC
:101E3000EE0FFF1FE657FC4F918380830F5F1F4F0C
:101E400082E090E0E80EF91E0D1518F3109273056C
:101E50001092E1058091E105882319F08F5F80934E
:101E6000E105DF91CF911F910F91FF90EF90DF90EF
:101E7000089510924A0410924F0410924E0410924A
:101E80005104109250040895882319F460E071E021
:101E900002C063E071E08FE796E00E94822C089513
:101EA000CF92DF92EF92FF921F93182F0E94452945
:101EB0009B01AC018091E2059091E305A091E405BE
:101EC000B091E50569017A01C81AD90AEA0AFB0A44
:101ED000D701C60189589341A040B04010F010923C
:101EE000E1052093E2053093E3054093E405509328
:101EF000E50590917405892F8150823020F4812F5F
:101F00000E944B0D0BC0933021F4812F0E94970D3E
:101F100005C0943019F4812F0E94A90E1F91FF90E3
:101F2000EF90DF90CF900895FF920F931F93CF9380
:101F3000DF93182F092FF62E8EE30E949F0A212F80
:101F4000302FC901EC0110E005C08FE769910E94B4
:101F50009F0A1F5F1F15C8F385E064E00E949F0A77
:101F600083E00E94990A8093420484E00E94990AC7
:101F7000809343040E944529609344047093450470
:101F8000809346049093470487E069E00E949F0A8B
:101F900081E08093FC03DF91CF911F910F91FF901F
:101FA00008950E94940F8091FC038130D9F40E941F
:101FB00045292091440430914504409146045091B4
:101FC0004704621B730B840B950B605A7648814063
:101FD000904040F4E8CF8FE796E067E071E00E9420
:101FE000822C08958091FC038130A9F308958FE736
:101FF00096E06EE70E944B2E0895BF92CF92DF923B
:10200000EF92FF920F931F93CF93DF936C018FE7B3
:1020100096E06EE70E944B2E760100E010E0C0E0F3
:10202000D0E080E2B82E0AC00830110521F49E01EC
:102030002095F60120870894E11CF11CF7016081CE
:10204000862F8D57823040F48FE796E06DE70E942F
:102050004B2EF70160816B258FE796E00E944B2E97
:102060000115110551F0F70180819E01280F311DE6
:10207000C32FDD27C20FD31FD0700F5F1F4F093052
:10208000110591F6DF91CF911F910F91FF90EF9085
:10209000DF90CF90BF900895DF93CF93CDB7DEB799
:1020A00029970FB6F894DEBF0FBECDBF382FE62FAD
:1020B0008091580590E0019664E270E00E94FE2E47
:1020C000982F8093580588E9898380E18A8391302D
:1020D00071F0913028F0923099F09330E1F416C00D
:1020E00085E08B8381EF8C832F5F2D8317C09B83CB
:1020F00081EF8C8384E6489FC00111249D830EC02C
:1021000084E08B8381EF8C833D8308C09B8381EFC8
:102110008C83ED8303C00E94F70F04C0CE010196AB
:102120000E94FD0F29960FB6F894DEBF0FBECDBFFB
:10213000CF91DF9108950F931F93CF93DF93182FC3
:10214000092F8FE796E06EE70E944B2E212F302F4C
:10215000C901EC0110E000E288818D57823040F423
:102160008FE796E06DE70E944B2E88818027888359
:102170008FE796E069910E944B2E1F5F193061F73F
:102180008FE796E06EE70E944B2EDF91CF911F9173
:102190000F910895DF93CF93CDB7DEB729970FB690
:1021A000F894DEBF0FBECDBF382F8091580588232D
:1021B00079F48EEF89833A836B83842F90E0959531
:1021C00087958C832D83198618861F821E822FC0C7
:1021D00040915305842F90E09C012F70307054E0A3
:1021E000959587955A95E1F78217930721F18DEF21
:1021F00089831A821B82DE01149620E008C0ED5B01
:10220000FA4F80818D93405F2F5F263069F0842FD5
:1022100090E0FC0134E0F595E7953A95E1F78F7091
:102220009070E817F90759F7409353052A83CE01B8
:1022300001960E949B108091580590E0019666E0FF
:1022400070E00E94FE2E8093580529960FB6F894F0
:10225000DEBF0FBECDBFCF91DF9108959F92AF92A9
:10226000BF92CF92DF92EF92FF920F931F93B82EFF
:10227000A62ED42EC22E902E0E9445297B018C01C1
:1022800080914205209154053091550540915605A5
:10229000509157058823B1F0D801C701821B930BD9
:1022A000A40BB50B815E9E42A040B04020F12C2DC6
:1022B000DC1408F42D2D8B2D6A2D422F292D0E9420
:1022C0004C1011C0D801C701821B930BA40BB50B96
:1022D00081539547A040B04070F08B2D6A2D4D2D55
:1022E0002C2D0E94CA10E0925405F09255050093DF
:1022F0005605109357051F910F91FF90EF90DF90B7
:10230000CF90BF90AF909F900895FF920F931F932F
:102310008C01F62E8FE796E00E944B2EF801848107
:102320008F2584831F910F91FF900895FF920F9343
:102330001F938C01F72E0E948511C8016F2D0E94FA
:1023400085111F910F91FF900895BF92CF92DF9258
:10235000EF92FF920F931F937C01B62E6A010FE755
:1023600016E0C80165EB0E944B2EC80162E60E9490
:102370004B2EF7011482C7016B2D0E948511C701F6
:10238000B6010E9496111F910F91FF90EF90DF9080
:10239000CF90BF9008958CE060E00E94CC298BE044
:1023A00061E00E94CC298DE061E00E94CC2982E0AE
:1023B00060E00E94CC2984E061E00E94CC2908956D
:1023C00082E08093B00085E08093B10083E061E01B
:1023D0000E94CC2983E060E00E94382A08951F9370
:1023E000182F0E94452960935405709355058093DA
:1023F00056059093570510934205112329F440E8A0
:1024000055E260E070E004C040E051EE60E070E052
:102410008FE796E00E94512D1F910895AF92BF92D1
:10242000CF92DF92EF92FF920F931F93DF93CF93A0
:10243000CDB7DEB76C970FB6F894DEBF0FBECDBF39
:102440000E9445297B018C0181E00E94810BF4E709
:10245000AF2E6E010894C11CD11CE3E0BE2EA982F0
:10246000C60161E00E94D10FB092FC030E94600C93
:102470006AEF70E080E090E00E946B298091FC039D
:10248000833009F08AC08FE796E00E94D82D892B0F
:1024900009F083C00E9445296E197F09800B910BBA
:1024A0006058734C894C914008F077C0D8CF8FE7C3
:1024B0000E94750A0E94890A843509F05CC08983EC
:1024C0000E94890A182F00E01093410500934005EF
:1024D0000E94890A080F111D1093410500934005C1
:1024E0000E94890A80933F050E94890A80933E05D5
:1024F000813108F040C0FF2407C00E94890A025EB3
:102500001A4FF8018083F3940F2D10E080913E055F
:1025100090E0880F991F0817190778F380E78983DF
:10252000CE01019661E00E94D10F83E08093FC030D
:102530000E94600C62E370E080E090E00E946B29F2
:102540008091FC038330A9F08FE70E94750A0E94F6
:10255000890A803581F4898307E214E00E94890AA0
:10256000F80181938F01F4E002341F07B9F781E08D
:1025700003C082E001C083E06C960FB6F894DEBF22
:102580000FBECDBFCF91DF911F910F91FF90EF90C4
:10259000DF90CF90BF90AF9008958091FC0383307F
:1025A00009F085CFE6CF83E00E94990A8093420428
:1025B00084E00E94990A8093430487E061E00E94CE
:1025C0009F0A6AE070E080E090E00E946B290E9420
:1025D000600C000008950F931F93082F17C05E9A98
:1025E00064E670E080E090E00E946B295E9864E60B
:1025F00070E080E090E00E946B291F5F101778F375
:102600006CE271E080E090E00E946B2910E0F6CF70
:10261000482F392F25E00DC0F999FECF1FBA842F1E
:10262000932F92BD81BD60BD0FB6F894FA9AF99AC6
:102630000FBE215059F0F999FECF842F932F92BDF0
:1026400081BDF89A80B5681739F7089582E00E9435
:10265000EB120895CF92DF92EF92FF920F931F93A8
:10266000CF93DF93C0E0D0E008E110E08EE1C82E08
:102670008EEBD82E81ECE82E8EEDF82E809126047C
:1026800090E00496B6E0880F991FBA95E1F7A7018C
:102690009601002E04C056954795379527950A94C4
:1026A000D2F78C0F9D1F622F0E94081321960850AD
:1026B0001040C430D10511F7C0E0D0E0809126046D
:1026C00090E0A6E0880F991FAA95E1F78C5F9E4FD6
:1026D000FE01E350FC4F8C0F9D1F60810E94081388
:1026E0002196C932D10551F7DF91CF911F910F91FA
:1026F000FF90EF90DF90CF90089580E490E060919C
:1027000026040E9408130895F999FECF80E490E012
:1027100092BD81BDF89A80B580932604843020F064
:10272000109226040E947D1308951F93182F0E9473
:10273000841380912604811731F0143020F4109313
:1027400026040E947D131F91089580915A058130BF
:10275000D1F0813020F0823009F043C037C08EE0E4
:102760000E946B2A892B09F03CC081E080935A05B6
:102770000E94372960935B0570935C0580935D052B
:1027800090935E0508958EE00E946B2A892BD9F400
:102790000E94372920915B0530915C0540915D05D1
:1027A00050915E05621B730B840B950B695E734041
:1027B00080409040B0F082E080935A0580ED97E031
:1027C0000E94D807089510925A0508958EE00E943D
:1027D0006B2A892B31F080E090E00E94D80710929C
:1027E0005A050895AF92BF92CF92DF92EF92FF9277
:1027F0000F931F93CF93DF938CE00E94990A882355
:10280000B9F58FE796E063E171E00E94822C5E9A51
:1028100080E00E94810B0E94600C5E9829C080912C
:102820007405882339F08FE796E00E94122E0E94EB
:10283000500F1EC08091DF05C82FD0E09E012F5F92
:102840003F4F2F7130708091DE0590E028173907D7
:1028500079F08FE796E00E94122ECB54DA4F8883EE
:102860008091DF0590E001968F7190708093DF0575
:102870008FE796E00E94D82D892B89F68091FC0382
:10288000843009F08CC00E944529609363057093E1
:102890006405809365059093660561157105810552
:1028A000910561F481E090E0A0E0B0E080936305E1
:1028B00090936405A0936505B093660580916F05BC
:1028C0009091700581609093700580936F0583E00F
:1028D0008093FC038FE70E94750ACCEAD5E00E9442
:1028E000890A899305E0C53BD007C9F74091970550
:1028F0008091AC05282F30E0842F90E08227932729
:1029000086FF40C080E4482740939705C90188733B
:102910009070C89709F510E014C01F5F80912504DE
:10292000E12FF0E084FF06C0E455FA4F80810E9459
:10293000830C07C0E455FA4F8FE796E060810E9450
:102940004B2E212F30E08091AC0590E08770907085
:102950008217930714F716C02F733070232B91F44E
:102960008091AD05809367058091AE0580936905E0
:102970008091AF0580936A058091B20580937105BF
:10298000109272058091E005813019F482E0809305
:10299000E0058091E005833011F41092E0050E947B
:1029A00045295B016C0180916B0590916C05A091AC
:1029B0006D05B0916E050097A105B105C9F0A6019E
:1029C0009501281B390B4A0B5B0BDA01C901885BA7
:1029D0009B40A040B04060F00E94C00A8093680510
:1029E00010926B0510926C0510926D0510926E0599
:1029F0008DEF93E00E94DC0820915F053091600527
:102A0000409161055091620586017501E21AF30A51
:102A1000040B150BE616F7060807190708F4E9C0BA
:102A2000A0925F05B0926005C0926105D0926205E8
:102A300080917305883008F0D4C0809173058F5F52
:102A400080937305E0906305F0906405009165053F
:102A500010916605E114F1040105110511F18DEFE6
:102A600093E00E94DC08AE18BF08C00AD10A6A15BC
:102A70007B058C059D0588F48091250485FD04C0A7
:102A800080ED97E00E94D8071092630510926405CC
:102A9000109265051092660504C080E090E00E94E7
:102AA000D80790919705907C909397050091DF054A
:102AB0001091DE050117B1F18091E005823091F5AA
:102AC0009058909397058DEF93E00E94D20889303B
:102AD00010F048E002C0482F415030E013C03F5F83
:102AE000A32FB0E0812F90E0FC01EB54FA4F20813E
:102AF000FD01E956FA4F2083AB52BA4F2C93019651
:102B0000182F1F71341710F4101749F71093DE05B2
:102B1000832F895C90919705892B8093970530933B
:102B2000D5051AC02091E0052430D1F49091D50547
:102B3000E6EDF5E0A8E9B5E0292F30E02E0F3F1FC4
:102B400002C081918D93E217F307D9F7995C8091C8
:102B50009705982B9093970583E08093E00523C019
:102B600080915A05823029F49160909397055E9A7E
:102B70000FC0909397055E98222319F481E080930B
:102B8000E0058091E005833019F484E08093E0054E
:102B9000F8948091250487706AE873E048E955E06D
:102BA0000E94630978945D9A809159050E94AA0A4F
:102BB0008DEF93E00E94D208682F87E995E00E948C
:102BC000940FE0915905EF5FE0935905E83131F03A
:102BD000F0E0E350FC4F8785882359F410925905A3
:102BE00008C080917305883009F45E9A89E080936B
:102BF000730580912504887171F18091FC03823006
:102C000051F580916F0590917005880F991F9093F1
:102C1000700580936F0583E08093FC030E94600C35
:102C20000E94452960936B0570936C0580936D0538
:102C300090936E05611571058105910561F481E040
:102C400090E0A0E0B0E080936B0590936C05A093BA
:102C50006D05B0936E058091250484FF1EC08091A0
:102C60006F05909170058E7F0E94000A182F809149
:102C70006705609171050E94400D082F80916805DD
:102C8000612F0E94400D282F8091690560916A058F
:102C9000402F009126040E942E115D980E94A513DA
:102CA000DF91CF911F910F91FF90EF90DF90CF9028
:102CB000BF90AF90089510921C0585E6E7EBF4E015
:102CC000DF011D928A95E9F708951F93182F8F371A
:102CD00019F0883009F042C0E0911C05EE2309F498
:102CE0005EC0E150E0931C05F0E0E954FB4F108218
:102CF0008FE796E06DE00E944B2E10E00DC0E12FB3
:102D0000F0E0E954FB4F6081772767FD70958FE70E
:102D100096E00E944B2E1F5F80911C05181778F3D8
:102D20008FE796E060E20E944B2E8FE796E06DE021
:102D30000E944B2E10E00DC0E12FF0E0E954FB4F54
:102D40006081772767FD70958FE796E00E944B2E94
:102D50001F5F80911C05181778F31FC08B3119F481
:102D60000E945B1622C08D3001F18A30F1F0809113
:102D70001C058436A0F4612F772767FD70958FE7D7
:102D800096E00E944B2E80911C05E82FF0E0E9545C
:102D9000FB4F10838F5F80931C0580E007C08FE797
:102DA00096E067E00E94E82AF8CF81E01F9108953D
:102DB0001F93CF93DF93CCE0D4E010E03BC08FE7CC
:102DC00096E062E271E00E947F2C8FE796E0612F2F
:102DD0004AE050E00E94F62B8FE796E06FE271E048
:102DE0000E947F2C699170E080E090E020910B04BC
:102DF00030E040E050E00E94DF2E20E137E240E08A
:102E000050E00E94DF2EDC01CB0140910204509182
:102E100003046091040470910504480F591F6A1F50
:102E20007B1F8FE796E02AE030E00E94BD2B1F5FFA
:102E3000183119F08881882311F6DF91CF911F9105
:102E40000895EF92FF920F931F93882339F48FE731
:102E500096E068E07AE00E94062B3BC090E00E947A
:102E6000990824E630E040E050E00E94112F122F34
:102E7000032FF42EE52E622F732F842F952F2AE037
:102E800030E040E050E00E94112F8FE796E0BA0159
:102E9000A9012AE030E00E94AE2B8FE796E06EE2B7
:102EA0000E94E82A612F702F8F2D9E2D2AE030E09E
:102EB00040E050E00E94112FAB01BC018FE796E08B
:102EC0002AE030E00E94AE2B8FE796E063E70E9495
:102ED0001A2B1F910F91FF90EF900895FF920F937F
:102EE0001F93CF93DF938FE796E06EEF79E00E9418
:102EF000C52A80912704813041F48FE796E065EE82
:102F000079E00E94062BFF2466C0823029F48FE707
:102F100096E06EEC79E0F5CF8430A9F78FE796E084
:102F20006AEB79E0EECFCF2DD0E0C930D1051CF0AF
:102F30006F2D685C02C06F2D6F5C8FE796E00E947A
:102F4000E82A8FE796E062EB79E00E94C52ABE018D
:102F50006F5F7F4F8FE796E04AE050E00E94582C69
:102F60008FE796E067EA79E00E94C52A8E01095D45
:102F70001B4FD8011196EC91E032F8F48FE796E000
:102F80006AE979E00E94C52AF8018181803130F038
:102F90008FE796E063E371E00E947F2CC95DDB4F11
:102FA000698170E06F7070706F5F7F4F8FE796E0A0
:102FB0004AE050E00E946B2C0DC0F0E0EF70F07022
:102FC000EE0FFF1FE555FC4F608171818FE796E0A2
:102FD0000E94822CF39480913F05F81608F4A3CF49
:102FE0008FE796E06FE779E00E94C52A80913F0461
:102FF0000E9421178FE796E064E679E00E94C52AD7
:10300000809140040E9421178FE796E069E479E0FF
:103010000E94C52A809141040E9421178FE796E003
:103020006EE279E00E94C52A40913704509138043D
:103030006091390470913A0441155105610571059B
:1030400039F18FE796E02AE030E00E94BD2B8FE750
:1030500096E06BEF78E00E94C52A80913B040E94C5
:10306000CC08AB01BC018FE796E02AE030E00E947B
:10307000BD2B8FE796E067ED78E00E94C52A8FE7C9
:1030800096E060913C044AE050E00E94082C06C0A3
:103090008FE796E06EEC78E00E94062B8FE796E0D3
:1030A00061EB78E00E94C52A60913D0470913E0476
:1030B0008FE796E04AE050E00E94E22B8FE796E02F
:1030C00064E978E00E94C52A60913604603150F4CA
:1030D00070E06F5F7F4F8FE796E04AE050E00E941C
:1030E0006B2C06C08FE796E06BE878E00E94062B19
:1030F0008FE796E06EE678E00E94C52A809135045D
:1031000080FD03C065E371E002C069E371E08FE711
:1031100096E00E94822C8FE796E061E578E00E94BD
:10312000C52A8091350482700E94440F8FE796E093
:1031300062E378E00E94C52A8091350484700E9481
:10314000440F8FE796E063E178E00E94C52A809102
:10315000350488700E94440FDF91CF911F910F9129
:10316000FF9008951F93CF93DF938FE796E062E57A
:103170007BE00E94C52A40910204509103046091B3
:103180000404709105048FE796E02AE030E00E9485
:10319000BD2B8FE796E06CE37BE00E94C52A40914F
:1031A00006045091070460910804709109048FE7A8
:1031B00096E020E130E00E94BD2B8FE796E066E2CA
:1031C0007BE00E94C52A8FE796E060910A044AE0FE
:1031D00050E00E94082C8FE796E060E17BE00E94BF
:1031E000C52A8FE796E060910B044AE050E00E9408
:1031F000082C8FE796E06AEF7AE00E94C52ACCE0BF
:10320000D4E010E012C0112331F08FE796E06DE3B7
:1032100071E00E947F2C8FE796E069914AE050E0D0
:103220000E94F62B1F5F183119F08881882359F707
:103230008FE796E00E94F02A8FE796E064EE7AE04E
:103240000E94C52A8FE796E0609124044AE050E08E
:103250000E94082C8FE796E06FEC7AE00E94C52A66
:10326000E0912504F0E0E770F070EE0FFF1FE553EA
:10327000FC4F608171818FE796E00E94822C8FE77E
:1032800096E06AEB7AE00E94C52A8091250490E0DE
:10329000887190708830910589F0893091051CF40F
:1032A000892B39F01BC08031910569F04897B1F442
:1032B0000FC08FE796E061EB7AE00EC08FE796E0F3
:1032C00065EA7AE009C08FE796E06FE97AE004C02A
:1032D0008FE796E065E97AE00E94062B8FE796E09B
:1032E00061E87AE00E94C52A4091FE035091FF03F5
:1032F00060910004709101048FE796E02AE030E0CD
:103300000E94BD2B8FE796E068E67AE00E94C52A0E
:103310008091250480720E94440F8FE796E06FE44D
:103320007AE00E94C52A8091250480740E94440F8F
:103330008FE796E066E37AE00E94C52A8091250433
:1033400080780E94440F8FE796E069E17AE00E945E
:10335000C52A8DEF93E00E94DC08AB01BC018FE72A
:1033600096E02AE030E00E94AE2B8FE796E064E121
:103370007AE00E94C52A8DEF93E00E94DC089B0151
:10338000AC0160E472E48FE090E00E94112F8FE7BF
:1033900096E0BA01A9012AE030E00E94AE2B8FE747
:1033A00096E061E17AE00E94062BDF91CF911F91B8
:1033B0000895EF92FF920F931F937C010FE716E0A1
:1033C000C8016F2D70E04AE050E00E94D12BC80187
:1033D0006EE20E94E82AB70154E0769567955A9507
:1033E000E1F76F707070C8014AE050E00E94D12B85
:1033F000C8016EE20E94E82A8FE0E822FF24C8019B
:10340000B7014AE050E00E94D12B1F910F91FF902D
:10341000EF9008950F931F93CF93DF932091B604FD
:103420002F3FA9F58FE796E063E975E00E94C52A72
:1034300084E593E00E94D9198FE796E062E775E092
:103440000E94C52A80914005909141050E94D9199A
:103450008FE796E06FE375E00E94062B8FE796E01A
:103460006CE175E00E94062B8FE796E064E075E062
:103470000E94062B8FE796E06FED74E00E94062B0A
:103480008FE796E00E94F02A0E946E1769C012161C
:103490000CF066C0332727FD309580913F0590E002
:1034A000821793070CF45CC08FE796E06AEC74E037
:1034B0000E94C52A6091B604772767FD70958FE753
:1034C00096E04AE050E00E946B2C8FE796E06FE9AF
:1034D00074E00E94C52A08E210E03AC0C12FD0E093
:1034E000CC0FDD1FC25EDA4F288130E08091B60438
:1034F000992787FD909501972817390741F58FE7A0
:1035000096E06FE371E00E947F2C8FE796E0602FDA
:103510004AE050E00E94F62B8FE796E063E471E00A
:103520000E947F2CE981F0E0EF70F070EE0FFF1F3A
:10353000E555FC4F608171818FE796E00E947F2CFA
:103540008FE796E067E471E00E947F2C0F5F1F5FBA
:1035500080913E05181710F28FE796E00E94F02A3E
:10356000DF91CF911F910F910895CF92DF92EF924B
:10357000FF920F931F93DF93CF93CDB7DEB76C9776
:103580000FB6F894DEBF0FBECDBF282F8091B604D2
:103590008F3F09F050C1822F992787FD9095A92F61
:1035A000B92FFC013A97EF36F10508F03DC1EC5C0C
:1035B000FF4FEE0FFF1F0590F491E02D09948FE768
:1035C00096E069E471E0B4C08FE796E069E471E0E9
:1035D0000E94822C22C18FE796E065E571E00E948F
:1035E000822C85E78983DE011296E7E2F4E08BE125
:1035F00001900D928150E1F7CE0101966CE10E949D
:10360000D10F0E94600C83E08093FC0368EC70E0B3
:1036100080E090E00E946B298091FC03843009F0E7
:1036200003C18FE70E94750A0E94890A8983853544
:1036300009F0FAC08FE796E061E874E00E94062B7B
:103640008FE796E063E674E00E94062B8FE796E032
:1036500065E474E0B2C08FE796E06DE671E00E9429
:10366000822C89E68983CE01019661E00E94D10F08
:103670000E94600C83E08093FC0368EC70E080E0C3
:1036800090E00E946B298091FC03843009F0CCC04B
:103690008FE70E94750A0E94890A89838E010E5F56
:1036A0001F4FFDE1EF2EF12CEC0EFD1E0E94890A4A
:1036B000D8018D938D01AE15BF05C1F7A7E2B4E027
:1036C000FE0132968BE101900D928150E1F78981E4
:1036D000893409F0A9C08FE796E067E274E00E94A0
:1036E000062B8FE796E069E074E00E94062B8FE7D7
:1036F00096E06BEE73E061C08FE796E067E871E0FB
:103700000E94822C8EEF8093B6048EC020522750E8
:10371000422F4053242F332727FD309580913F05BA
:1037200090E0821793073CF48FE796E066E971E03A
:103730000E94822C79C04093B6046FC084E18093CC
:10374000B6048FE796E064EB73E037C085E18093C1
:10375000B6048FE796E06DE773E02FC086E18093B3
:10376000B6048FE796E066E473E027C087E18093B4
:10377000B6048FE796E06CEF72E01FC088E180939B
:10378000B6048FE796E06BEE72E017C089E1809394
:10379000B6048FE796E067ED72E00FC08AE1809390
:1037A000B6048FE796E062EC72E007C08BE180938D
:1037B000B6048FE796E06AE972E00E94062B34C0F7
:1037C0008FE796E060E872E00E94062B8091350456
:1037D00091E01DC08FE796E06AE672E00E94062B3A
:1037E0008091350492E013C08FE796E065E572E0C2
:1037F0000E94062B8091350494E009C08FE796E083
:103800006AE372E00E94062B8091350498E08927D4
:10381000809335048FEF8093B6040E940A1A04C087
:103820008FE796E00E94122E8FE796E00E94D82D37
:10383000892BB1F777C1822F0E946516882309F47E
:1038400071C180911C05882321F48FEF8093B60409
:1038500061C187EB94E060E070E040E050E00E94DE
:103860006E069B01AC019091B604963109F47CC0C0
:10387000973164F4943109F463C095310CF06AC057
:10388000892F81508D3008F035C113C0993109F46A
:10389000E5C09A313CF4973109F470C0983109F0D1
:1038A00029C1D2C09A3109F4E7C09B3109F022C185
:1038B000F5C0E92FFF27E7FDF09580913F0590E0E7
:1038C0008E179F070CF416C1DA01C9010197A109EF
:1038D000B1098097A105B10540F0FF2410E008E28E
:1038E0006F010894C108D10826C0E95DFB4F822F03
:1038F00081508083E7C0612F70E0660F771F625EA2
:103900007A4FFB01808190E08C159D0599F4802F02
:1039100090E0A0E0B0E082179307A407B50749F450
:10392000F601E95DFB4FDB0111968C918183FF2449
:10393000F3940F5F1F5F80913E051817E0F2C0C03F
:103940002F3F31054105510511F008F0D3C02093F8
:103950003F04B8C02F3F31054105510511F008F073
:10396000C9C020934004AEC02F3F31054105510529
:1039700011F008F0BFC020934104A4C08091B704A7
:103980008062803719F588EB94E060E070E040E0F9
:1039900050E00E946E069B01AC01DC01CB01019757
:1039A000A109B1090897A105B10508F0B6C0CA017F
:1039B000B90124ED30E340E050E00E94DF2E9B018E
:1039C000AC012A5E3C4A4A46554E24C0863611F563
:1039D00088EB94E060E070E040E050E00E946E060A
:1039E0009B01AC01DC01CB010197A109B10907974B
:1039F000A105B10508F091C0CA01B90128EA31E674
:103A000040E050E00E94DF2E9B01AC01245E3C436D
:103A10004E46544E211531054105510561F0DA013C
:103A2000C9018054914EAD49B8418158904FAA4F79
:103A3000B24008F05FC020933704309338044093BD
:103A4000390450933A043EC02F3F310541055105DA
:103A500011F008F04FC020933B0434C0DA01C901D3
:103A60000197A109B1098F3F9105A105B10508F0A2
:103A700041C020933C0426C0DA01C901845C99400E
:103A8000A040B0408D549D41A040B04038F43093E8
:103A90003E0420933D04FF24F39401C0FF2421152C
:103AA00031054105510511F48FEF07C02131310572
:103AB0004105510528F4822F81508093360402C0BD
:103AC000FF20C1F080911D058823D1F48091060468
:103AD00090910704A0910804B09109040196A11DDA
:103AE000B11D8093060490930704A0930804B0933B
:103AF000090406C08FE796E068EA71E00E94822C14
:103B00000E945B168FEF8093B6048FE796E06AE021
:103B10000E941A2B0E940A1A05C021E030E040E002
:103B200050E07DCF6C960FB6F894DEBF0FBECDBFD0
:103B3000CF91DF911F910F91FF90EF90DF90CF9089
:103B400008958FE796E06EEE71E00E94062B8FE7F6
:103B500096E066ED71E00E94062B8FE796E00E94EA
:103B6000D82D892B31F08FE796E00E94122E0E940B
:103B7000B51A0E940E12823019F0833069F405C024
:103B80008FE796E068EB71E004C08FE796E061EAAA
:103B900071E00E94062B08958FEF8093B604109277
:103BA0001D050E940A1A0CC08FE796E00E94D82DCE
:103BB000892B31F08FE796E00E94122E0E94B51AF1
:103BC0008091B6048E3F81F708958091B6048430C9
:103BD00009F46FC0853084F4813009F45BC0823011
:103BE00024F48F3F09F085C014C0823009F457C017
:103BF000833009F07EC058C0863009F464C0863036
:103C00000CF45CC0873009F463C0893009F071C0DE
:103C10006AC08FE796E066E078E00E94062B84E5B4
:103C200093E00E94D9198FE796E06EEE77E00E944C
:103C3000062B8FE796E069EC77E00E94062B8FE772
:103C400096E06FE977E00E94062B8FE796E06EE73B
:103C500077E00E94062B8FE796E061E577E00E940F
:103C6000062B8FE796E06BE277E00E94062B8FE74A
:103C700096E067E077E00E94062B8FE796E060EE23
:103C800076E00E94062B8FE796E00E94F02A0E94C1
:103C9000B2182FC08FE796E063EC76E028C08FE77C
:103CA00096E06EE976E023C08FE796E069E876E07B
:103CB0001EC08FE796E06AE676E019C08FE796E0CF
:103CC00066E276E014C08FE796E061E176E00FC02F
:103CD0008FE796E06CEF75E00E94062B8FE796E089
:103CE00066EB75E004C08FE796E060EA75E00E943D
:103CF000062B6AE070E080E090E00E946B2904C02F
:103D00008FE796E00E94122E8FE796E00E94D82D52
:103D1000892BB1F708952F923F924F925F926F9245
:103D20007F928F929F92AF92BF92CF92DF92EF924B
:103D3000FF920F93DF93CF93CDB7DEB7A8970FB65F
:103D4000F894DEBF0FBECDBF7E010894E11CF11CCC
:103D500080E1D7011D928A95E9F78FE796E066EC3E
:103D600071E00E94822C0E94D31220E431EE4DE9D2
:103D700058E129A33AA34BA35CA380EC91EDA8E9F9
:103D8000BBE18D8F9E8FAF8FB8A324EF31E040E071
:103D900050E0298F3A8F4B8F5C8FB0E58B2EB3ECC0
:103DA0009B2EA12CB12C80E491EEADE9B8E18D8B76
:103DB0009E8BAF8BB88F44245524320100E022241F
:103DC0003324198A1A8A1B8A1C8A0DC18FE796E050
:103DD0000E94122E8434C9F0853434F48332C9F140
:103DE0008C3209F0CEC046C0833509F0CAC029A183
:103DF0003AA14BA15CA1C901DA018D8B9E8BAF8BDF
:103E0000B88F442455243201EEC08FE796E064E475
:103E10000E94E82A8FE796E040E451EE6DE978E1F0
:103E20002AE030E00E941C2C8FE796E06CE20E94B2
:103E3000E82A8FE796E040EC51ED68E97BE12AE063
:103E400030E00E941C2C8FE796E06CE20E941A2B57
:103E5000CAC019821A821B821C821D821E821F8286
:103E6000188619861A861B861C861D861E861F8646
:103E7000188A3CC00F5F043009F0B5C069817A81AF
:103E80008B819C8128EE33E040E050E00E94DF2EE1
:103E900069A37AA38BA39CA36D817E818F81988572
:103EA0000E94DF2E6D8F7E8F8F8F98A329853A8594
:103EB0004B855C85298F3A8F4B8F5C8F6D857E8516
:103EC0008F85988928EE33E040E050E00E94DF2E95
:103ED0004B015C0160323EE4730730E0830730E061
:103EE000930730F48CE162E30E949F0A00E07BC0FC
:103EF000603345E7740740E0840740E0940718F416
:103F00008CE162E2F1CF60345CE9750750E085072F
:103F100050E0950718F48CE166E2E6CF80E588165C
:103F200083EC980680E0A80680E0B80618F48CE1DF
:103F300062E1DACF90E689169AEE990690E0A9063A
:103F400090E0B90618F48CE165E1CECFA0E78A16BF
:103F5000A1E19A06A1E0AA06A0E0BA0618F48CE155
:103F600061E0C2CFB0EA8B16B6E89B06B1E0AB06C3
:103F7000B0E0BB0618F48CE163E0B6CF8CE165E0FD
:103F8000B3CF80538A3078F5C02EDD24CC0CDD1CF5
:103F9000CC0CDD1CE1E0F0E0EC0FFD1FCE0EDF1ECF
:103FA000282F332727FD3095432F532F2DA33EA3D2
:103FB0004FA358A7D6016D917D918D919C912AE0D8
:103FC00030E040E050E00E94DF2E2DA13EA14FA145
:103FD00058A5260F371F481F591FD6012D933D9313
:103FE0004D935C9313978FE796E00E94D82D892B11
:103FF00009F0ECCE411451046104710499F46D8907
:104000007E898F89988D0E94150B61E070E080E0B9
:1040100090E00E946B2922242A943324198A1A8A58
:104020001B8A1C8A298D3A8D4B8D5C8D4216530656
:1040300064067506D0F40E94C00A29893A894B8922
:104040005C89280F311D411D511D298B3A8B4B8BEB
:104050005C8B381608F4382E821508F4282E089444
:10406000411C511C611C711C64C06D897E898F8943
:10407000988D28EE33E040E050E00E94112F8FE74A
:1040800096E0BA01A9012AE030E00E94AE2B8FE74A
:1040900096E06CE20E94E82A8FE796E0632D4AE002
:1040A00050E00E94F62B8FE796E06CE20E94E82A2F
:1040B00069897A898B899C89A30192010E94112FB9
:1040C0008FE796E0BA01A9012AE030E00E94AE2B0A
:1040D0008FE796E06CE20E94E82A8FE796E0622D77
:1040E0004AE050E00E94F62B8FE796E06CE20E94D7
:1040F0001A2B8D899E89AF89B88D880D991DAA1DAF
:10410000BB1D8D8B9E8BAF8BB88F2D8D3E8D4F8DB4
:1041100058A1281739074A075B0740F489A19AA1DB
:10412000ABA1BCA18D8B9E8BAF8BB88F4424552443
:10413000320129A13AA14BA15CA1285E3340404045
:10414000504009F050CFA8960FB6F894DEBF0FBECE
:10415000CDBFCF91DF910F91FF90EF90DF90CF9087
:10416000BF90AF909F908F907F906F905F904F9097
:104170003F902F900895CF92DF92EF92FF920F938E
:104180001F93DF93CF93CDB7DEB7E8970FB6F894C0
:10419000DEBF0FBECDBF7C01FC018281883009F4F7
:1041A000ABC08930A8F4843009F45FC0853048F48E
:1041B0008230E9F1833008F04DC0813009F080C1D0
:1041C00023C0863009F482C0873008F08BC060C0FD
:1041D000883609F4D4C0893650F4863609F4AFC065
:1041E000873608F0C5C0853609F06AC18FC08A36A7
:1041F00009F4FEC08A3608F4F2C08B3609F438C1DF
:10420000873C09F05DC149C1C70161E049E250E066
:104210000E94A5110DEF13E0C701F80161918F0114
:104220000E948511F4E006321F07B1F753C1C701A0
:1042300062E04BE150E00E94A51107E214E0C701E3
:10424000F80161918F010E948511F4E002341F078B
:10425000B1F740C1C70163E041E050E00E94A51101
:104260000E940E12682FC70133C1C70164E041E00C
:1042700050E00E94A511C70161E00E9485118FE7FF
:1042800096E0F70164810E944B2E0E948B1E28C18C
:1042900040913E0550E0440F551FC70165E00E9464
:1042A000A51100E010E009C0F801E25EFA4FC70175
:1042B00060810E9485110F5F1F4F80913E0590E045
:1042C000880F991F0817190778F304C1C70166E022
:1042D00042E050E00E94A511C70164E573E00E942E
:1042E0009611F8C0C70167E041E050E00E94A511B7
:1042F000C70160913F05ECC0C70168E041E050E0B4
:104300000E94A511C70160912604E2C0C70165E6BD
:1043100041E050E00E94A511F701878190858997BF
:1043200009F0D4C0D701EDEFF3E019968C911997FD
:104330008193119684E0E632F807B9F7ABC0C70164
:1043400066E641E050E00E94A511F7018781908563
:104350004B9709F0BBC0D701E7E2F4E019968C91C6
:1043600019978193119684E0E234F807B9F792C067
:10437000C70167E641E050E00E94A51189C0C7016E
:1043800068E641E050E00E94A51185E78983DE01DF
:104390001296E7E2F4E08BE101900D928150E1F793
:1043A000CE0101966CE10E94D10F0E94600C83E067
:1043B0008093FC0368EC70E080E090E00E946B2941
:1043C0008091FC03843009F081C08FE70E94750A58
:1043D0000E94890A8983853509F078C05BC0C701CE
:1043E00069E641E050E00E94A5110E94540852C0C5
:1043F000C7016AE641E050E00E94A51189E68D8F71
:10440000CE014D9661E00E94D10F0E94600C83E0C6
:104410008093FC0368EC70E080E090E00E946B29E0
:104420008091FC03843009F051C08FE70E94750A27
:104430000E94890A8D8F8E01025E1F4F89E3C82E6C
:10444000D12CCC0EDD1E0E94890AF80181938F01C8
:10445000EC15FD05C1F7A7E2B4E0FE017E968BE105
:1044600001900D928150E1F78D8D893479F512C05C
:10447000C7016BE641E050E00E94A511F70181857C
:104480000E9495130E940408892B21F40E9454086D
:104490000E942A13C70161E01BC0C70167EC41E01D
:1044A00050E00E94A511C70161E00E9485118FE7CD
:1044B00096E0F70164810E944B2E1092480410C0D0
:1044C000C7016AEC41E050E00E94A511C70160E01D
:1044D0000E9485118FE796E0F70164810E944B2EC0
:1044E000E8960FB6F894DEBF0FBECDBFCF91DF9137
:1044F0001F910F91FF90EF90DF90CF9008956F92F2
:104500007F928F929F92AF92BF92CF92DF92EF9263
:10451000FF920F931F93CF93DF9381E08093480422
:10452000BEE4EB2EB4E0FB2EA4E0CA2ED12CCE0CC0
:10453000DF1CF4E66F2EE4E07E2E76E0972E65E039
:10454000862E52E0A52E43E0B42EB8C08FE796E049
:104550000E94D82D892B09F4B1C0A9C08FE796E03D
:104560000E94122E982F8093490480914A04833030
:1045700021F1843028F4813099F08230B8F409C0F8
:10458000853009F450C0853020F1863009F08FC0A5
:1045900067C0953B09F08BC081E080934A0487C0D7
:1045A000923609F082C0A0924A0481C090934B04D5
:1045B00090934C04B0924A047AC090934E04F70151
:1045C000118280914C04892780934C0470924A0494
:1045D0006EC0D92FC0E020914E0430914F042C2B97
:1045E0003D2B30934F0420934E0480914C04892737
:1045F00080934C0480924A042536310508F457C054
:1046000089E494E06CEC41E050E00E94A51189E45B
:1046100094E061E00E9485118FE796E060914D047F
:104620000E944B2E42C02091500430915104F90158
:10463000E75BFB4F918780914C04892780934C0462
:104640002F5F3F4F309351042093500480914E04CC
:1046500090914F042817390750F190924A0427C0CF
:1046600000914C04091729F489E494E00E94BB20CE
:1046700013C010914B0489E494E06BEC42E050E0ED
:104680000E94A51189E494E0612F0E94851189E4BC
:1046900094E0602F0E948511F601862D11928A9573
:1046A000E9F7109251041092500410924A048FE7D7
:1046B00096E00E94D82D892B09F050CF80914804B4
:1046C000813009F443CFDF91CF911F910F91FF907B
:1046D000EF90DF90CF90BF90AF909F908F907F90A2
:1046E0006F900895DF92EF92FF920F931F93CF93F5
:1046F000DF930E9445296115710581059105C9F374
:104700000E94650610920604109207041092080495
:1047100010920904DD24E0900604F0900704009153
:10472000080410910904102F0F2DFE2CEE240E9476
:1047300060062FEF30E040E050E00E94332FE60E9D
:10474000F71E081F191FE0920604F0920704009359
:10475000080410930904D39484E0D816E1F6CCE061
:10476000D4E010E017C00E94600622E330E040E091
:1047700050E00E94332F6F5FECE0F4E090E004C063
:104780008191861781F39F5F9117D0F369931F5F23
:10479000183119F08881882331F7DF91CF911F916B
:1047A0000F91FF90EF90DF9008951F931091B60442
:1047B0001F3F09F0BFC0893409F466C08A342CF564
:1047C000883309F476C089336CF4803309F481C0EE
:1047D00081330CF06CC08B3109F44CC0813209F08C
:1047E000A3C03CC0813409F483C082343CF48933D3
:1047F00009F46DC0803409F097C030C0823409F4E8
:1048000082C0863409F090C04FC0823609F47BC064
:1048100083368CF4883571F1893534F48235E9F1C9
:10482000833509F081C01FC08A3509F478C081360C
:1048300009F07AC05DC0823781F1833734F486365F
:1048400099F1893609F070C01FC0883799F08A370E
:1048500009F465C0833709F067C005C08FE796E0AB
:1048600069E471E017C00E942A138FE796E063EDB8
:1048700071E006C00E9404088FE796E06DEE71E0DB
:104880000E94822C8EEF4EC00E9454088FE796E063
:104890006CE072E00E94822C47C00E9472238FE776
:1048A00096E065E272E0F6CF0E94D8163DC08053D4
:1048B00039C08FE796E06EE871E00E94062B909178
:1048C0002504892F885F8871977E892B0CC089E029
:1048D00029C08FE796E06BE771E00E94062B80917C
:1048E000250490E28927809325041093B6041CC008
:1048F0008FE796E065E671E00E94062B8091250423
:1049000090E4892709C08FE796E064E571E00E9492
:10491000062B8091250480588093250402C00E94B4
:10492000A11D8FEF8093B6048091B6048E3F09F4E9
:10493000E8C0DFC00E946516882309F4E2C08091B8
:104940001C05882321F48FEF8093B604D2C087EB37
:1049500094E060E070E040E050E00E946E069B0151
:10496000AC018091B604843009F441C0853044F430
:10497000823041F1833094F5813009F096C00DC04A
:10498000863009F467C086300CF43EC0873009F4E5
:1049900069C0893009F089C075C0DA01C901815444
:1049A000914EAD49B8418F57904FAA4FB24008F091
:1049B0007CC020930204309303044093040450937A
:1049C00005049AC02093060430930704409308041A
:1049D0005093090481E080931D058EC02830310575
:1049E0004105510508F061C020930A0485C0DA0131
:1049F000C9010197A109B1090A97A105B10508F0FC
:104A000054C020930B0478C087EB94E06DE371E011
:104A10000E948A0710E00EC0183130F4E12FF0E058
:104A2000E350FC4F87871F5F80E090E06DE371E00B
:104A30000E948A07009759F00E946C07009761F75F
:104A400006C0E12FF0E0E350FC4F17861F5F1831DE
:104A5000C0F352C0253031054105510530F5209392
:104A600024044AC0DA01C9010197A109B1090697D6
:104A7000A105B105D0F480912504887F822B809315
:104A800025043AC0DA01C9010197A109B109805092
:104A9000924CA140B04048F42093FE033093FF03B2
:104AA000409300045093010427C08FE796E068EA22
:104AB00071E00E94822C13C080910604909107043B
:104AC000A0910804B09109040196A11DB11D809325
:104AD000060490930704A0930804B09309040E946D
:104AE0005B168FEF8093B6048FE796E06AE00E9432
:104AF0001A2B0E94E51D05C080911D058823E1F257
:104B0000EECF1F9108958FEF8093B60410921D058C
:104B10000E94E51D0CC08FE796E00E94D82D892BDE
:104B200031F08FE796E00E94122E0E94D5238091EB
:104B3000B6048E3F81F76AE070E080E090E00E946A
:104B40006B2904C08FE796E00E94122E8FE796E053
:104B50000E94D82D892BB1F708957F928F929F9252
:104B6000AF92BF92CF92DF92EF92FF920F931F937B
:104B7000DF93CF93CDB7DEB7AA970FB6F894DEBF19
:104B80000FBECDBF0E9437296B017C0181E00E94DE
:104B9000810B04C08FE796E00E94122E8FE796E00B
:104BA0000E94D82D892BB1F75E9811E022E6722E73
:104BB00092E0892E912C8C0E9D1E5E010894A11C02
:104BC000B11C03E00E94372920E030E06C197D0918
:104BD0008E099F09693C71058105910510F021E05E
:104BE00030E0812F90E028233923232BA9F10E9464
:104BF00037296B017C015D9A80ED97E00E94D80710
:104C00007982D401EDEFF3E089E201900D928150B9
:104C1000E1F7C5016AE20E94D10F5D9880E090E063
:104C20000E94D8070093FC030E94600C62E370E0CE
:104C300080E090E00E946B298091FC03843059F45D
:104C40000093FC038FE70E94750A0E94890A823450
:104C500011F410E001C011E08EE00E946B2A892B54
:104C600041F511E026C05E9A5D9A8FE796E00E94BA
:104C7000122E8D30910569F08E3091051CF40A9743
:104C8000B1F407C08332910569F08234910579F45B
:104C90000CC08FE796E066E471E00E94062B0E944C
:104CA000832505C00E948B1E02C00E947F225E9851
:104CB0005D988FE796E00E94D82D892B09F482CF6A
:104CC000D2CF8FE796E00E94D82D04970CF18FE7A2
:104CD00096E00E94122E82349105D1F48FE796E07F
:104CE0000E94122E8E34910599F48FE796E00E946F
:104CF000122E8434910561F48FE796E00E94122E03
:104D0000819731F480E090E00E94D8070E94AD25A1
:104D100008958F929F92AF92BF92CF92DF92EF92BF
:104D2000FF920F931F938EE00E946B2A892B09F04C
:104D3000ACC068EC70E080E090E00E946B2980E0FD
:104D400090E00E94D8070E9437295B016C0130EC8B
:104D5000E32E32E1F32E012D112DE60EF71E081F72
:104D6000191F06C08EE00E946B2A892B09F085C0AE
:104D70000E9437296E157F058007910798F38EE012
:104D80000E946B2A892B09F078C080ED97E00E9481
:104D9000D8070E9437297B018C0199249394882499
:104DA00088E496E2A0E0B0E0A80EB91ECA1EDB1EA1
:104DB00029C0AE14BF04C006D10638F480ED97E0D8
:104DC0000E94D807882483941DC00E9437296E1939
:104DD0007F09800B910B693C71058105910590F06D
:104DE0000E9437297B018C0180E0992009F481E041
:104DF000982E882319F480E090E002C080ED97E0BF
:104E00000E94D8078EE00E946B2A892B91F280E0E5
:104E100090E00E94D807882051F1809126048F5F8E
:104E200083700E9495138FE796E062E472E00E941F
:104E30007F2C8FE796E0609126044AE050E00E94C4
:104E4000082C0E940408892B39F08FE796E06FE464
:104E500072E00E94822C19C08FE796E06CE672E047
:104E60000E947F2C0E9454080E942A130EC00E94A8
:104E700072230E942A130E94B2188FE796E06EE810
:104E800072E00E94822C0E94AD251F910F91FF902D
:104E9000EF90DF90CF90BF90AF909F908F9008954C
:104EA00080E069EC77E042E050E00E9472280895CB
:104EB000EF92FF920F931F930E94CB1189E061E064
:104EC0000E94CC2989E060E00E94382A86E061E0F7
:104ED0000E94CC2985E061E00E94CC298EE060E050
:104EE0000E94CC2988E060E00E94CC2988E061E043
:104EF0000E94382A81E161E00E94CC2981E160E0D2
:104F00000E94382A0E94E0118FE796E040E052ECC0
:104F100061E070E00E94512D0E9484130E940408F9
:104F2000892B39F08FE796E06FE472E00E94822CC3
:104F30000AC08FE796E06CE672E00E947F2C0E9428
:104F400054080E942A130E94250D8FEF8093730549
:104F50000E94502778940E9437297B018C01809110
:104F600073058F3F09F0AFC00E9437296E197F0982
:104F7000800B910B605D77408040904008F0A3C0AB
:104F8000EECF8FE796E00E94122E8FE796E00E9408
:104F9000D82D892BB1F78FE796E065EA72E00E9481
:104FA0007F2C84E593E00E94D9198FE796E06CEBA3
:104FB00072E00E947F2C8FE796E064E070E04AE0A8
:104FC00050E00E946B2C68EC70E080E090E00E9462
:104FD0006B290E9461264091FE035091FF0360916E
:104FE000000470910104DB01CA010197A109B10914
:104FF0000497A105B10568F440937405433029F086
:1050000040E052EC61E070E004C040EA56E861E044
:1050100070E08FE796E00E94512D0E9489265E98ED
:1050200080E090E00E94D8070E94250D80E00E9459
:10503000810B809159050E94AA0A0E94600C10926F
:10504000DE051092DF051092E0056CE271E080E071
:1050500090E00E946B2980ED97E00E94D80764E6FB
:1050600070E080E090E00E946B2980E090E00E9478
:10507000D80710E015C064E670E080E090E00E9480
:105080006B2980ED97E00E94D80764E670E080E02D
:1050900090E00E946B2980E090E00E94D8071F5F9B
:1050A00080912604181738F38091250490E084FF3E
:1050B00014C020E088719070489709F421E0822F95
:1050C0000E94EF110AC080ED97E00E94D8078EE0A1
:1050D00061E00E94382A5E9A58CF1F910F91FF908D
:1050E000EF900895823000F5E82FF0E0EE0FFF1FFB
:1050F000E651FA4F71836083882319F08130A1F45F
:1051000008C0809169008C7F842B80936900E89AA5
:10511000089580916900440F551F440F551F837FE8
:10512000842B80936900E99A08951F920F920FB61D
:105130000F9211242F933F934F935F936F937F931D
:105140008F939F93AF93BF93EF93FF938091EA0563
:105150009091EB05892B29F0E091EA05F091EB05A0
:105160000995FF91EF91BF91AF919F918F917F91A1
:105170006F915F914F913F912F910F900FBE0F90C4
:105180001F9018951F920F920FB60F9211242F9314
:105190003F934F935F936F937F938F939F93AF93BF
:1051A000BF93EF93FF938091EC059091ED05892BD0
:1051B00029F0E091EC05F091ED050995FF91EF9153
:1051C000BF91AF919F918F917F916F915F914F911F
:1051D0003F912F910F900FBE0F901F9018951F9227
:1051E0000F920FB60F9211242F933F938F939F939B
:1051F000AF93BF938091F2059091F305A091F405D0
:10520000B091F5053091F6050196A11DB11D232F32
:105210002D5F2D3720F02D570196A11DB11D209334
:10522000F6058093F2059093F305A093F405B093EF
:10523000F5058091EE059091EF05A091F005B091F4
:10524000F1050196A11DB11D8093EE059093EF0528
:10525000A093F005B093F105BF91AF919F918F910D
:105260003F912F910F900FBE0F901F9018958FB701
:10527000F8942091F2053091F3054091F405509196
:10528000F5058FBFB901CA0108959FB7F894209121
:10529000EE053091EF054091F0055091F10586B58E
:1052A000A89B06C08F3F21F02F5F3F4F4F4F5F4FAE
:1052B0009FBF542F432F322F2227280F311D411D0E
:1052C000511D82E0220F331F441F551F8A95D1F7CD
:1052D000B901CA010895EF92FF920F931F93CF93E4
:1052E000DF937B018C010E944529EB010EC00E94D7
:1052F00045296C1B7D0B685E7340C8F30894E10878
:10530000F10801091109C851DC4FE114F10401054C
:10531000110569F7DF91CF911F910F91FF90EF90E9
:105320000895789484B5826084BD84B5816084BD1D
:1053300085B5826085BD85B5816085BDEEE6F0E00E
:10534000808181608083E1E8F0E01082808182606A
:105350008083808181608083E0E8F0E080818160EB
:105360008083E1EBF0E0808184608083E0EBF0E01B
:10537000808181608083EAE7F0E0808184608083BF
:105380008081826080838081816080838081806869
:1053900080831092C1000895CF93DF93482F50E08F
:1053A000CA018656944FFC0134914A57544FFA0172
:1053B0008491882369F190E0880F991FFC01E859D6
:1053C000F44FA591B491FC01EE58F44FC591D491DE
:1053D000662351F42FB7F8948C91932F90958923DD
:1053E0008C93888189230BC0623061F42FB7F894C5
:1053F0008C91932F909589238C938881832B88831C
:105400002FBF06C09FB7F8948C91832B8C939FBFBE
:10541000DF91CF910895833071F0843028F481308A
:10542000A1F0823021F514C08630B1F08730D1F080
:105430008430E9F404C0809180008F7703C08091AC
:1054400080008F7D80938000089584B58F7702C09F
:1054500084B58F7D84BD08958091B0008F7780934F
:10546000B00008958091B0008F7D8093B0000895C2
:10547000FF920F931F93F62E482F50E0CA018255DA
:10548000944FFC012491CA018656944FFC0114915B
:105490004A57544FFA0104910023C9F0222319F00E
:1054A000822F0E940B2AE02FF0E0EE0FFF1FEE5834
:1054B000F44FA591B4919FB7F894FF2021F48C91FB
:1054C0001095812302C08C91812B8C939FBF1F91DB
:1054D0000F91FF9008950F931F93482F50E0CA013A
:1054E0008255944FFC012491CA018656944FFC01C9
:1054F00004914A57544FFA011491112319F420E0F2
:1055000030E015C0222319F0822F0E940B2A812F30
:1055100090E0880F991F8458944FFC01A591B49195
:105520008C9120E030E0802311F021E030E0C901CF
:105530001F910F910895CF92DF92EF92FF920F93F8
:105540001F93CF93DF937C016B018A01C0E0D0E011
:105550000FC0D6016D916D01D701ED91FC910190C5
:10556000F081E02DC7010995C80FD91F01501040E7
:105570000115110571F7CE01DF91CF911F910F91A8
:10558000FF90EF90DF90CF900895EF92FF920F93EE
:105590001F93CF93DF937C018B01C0E0D0E0F80133
:1055A0000F5F1F4F6491662359F0D701ED91FC9175
:1055B0000190F081E02DC7010995C80FD91FEFCFE9
:1055C000CE01DF91CF911F910F91FF90EF90089541
:1055D000DC01ED91FC910190F081E02D0995089599
:1055E000EF92FF920F931F938C016DE00E94E82AC7
:1055F0007C01C8016AE00E94E82A9C012E0D3F1D33
:10560000C9011F910F91FF90EF900895EF92FF92C3
:105610000F931F937C010E94C52A8C01C7010E9431
:10562000F02A9C01200F311FC9011F910F91FF909B
:10563000EF900895EF92FF920F931F937C010E94C9
:10564000E82A8C01C7010E94F02A9C01200F311F1B
:10565000C9011F910F91FF90EF900895CF93DF93B1
:10566000EC016115710519F420E030E00FC0DB0199
:105670000D900020E9F71197A61BB70BE881F9817F
:105680000280F381E02DAD0109959C01C901DF91F4
:10569000CF9108954F925F927F928F929F92AF9297
:1056A000BF92CF92DF92EF92FF920F931F93DF93FF
:1056B000CF93CDB7DEB7A1970FB6F894DEBF0FBE7C
:1056C000CDBF2C01742ECB01223008F42AE019A2A0
:1056D00031E2C32ED12CCC0EDD1E822E9924AA24B9
:1056E000BB24672D752FA50194010E94112F79010C
:1056F0008A01C801B701A50194010E94DF2E472D40
:10570000461B0894C108D1084A3014F4405D01C01A
:10571000495CF6014083E114F1040105110521F013
:105720007E2C5F2DC801DDCFC201B6010E942E2B59
:10573000A1960FB6F894DEBF0FBECDBFCF91DF911B
:105740001F910F91FF90EF90DF90CF90BF90AF909F
:105750009F908F907F905F904F900895DC0121156E
:10576000310541F4ED91FC910190F081E02D642F21
:10577000099508950E944A2B0895EF92FF920F9386
:105780001F937C010E94AE2B8C01C7010E94F02A5E
:105790009C01200F311FC9011F910F91FF90EF90C5
:1057A0000895EF92FF920F931F939A017B0100E0FF
:1057B00010E0B801A7010E94AE2B1F910F91FF903E
:1057C000EF900895EF92FF920F931F937C010E9438
:1057D000D12B8C01C7010E94F02A9C01200F311FA0
:1057E000C9011F910F91FF90EF900895EF92FF92E2
:1057F0000F931F939A01E62EFF2400E010E0B801FA
:10580000A7010E94AE2B1F910F91FF90EF9008957A
:10581000EF92FF920F931F937C010E94F62B8C0155
:10582000C7010E94F02A9C01200F311FC9011F915E
:105830000F91FF90EF900895CF92DF92EF92FF9239
:105840000F931F93CF93DF93EC016A017B01211526
:10585000310541F4E881F9810190F081E02D642F58
:1058600009951BC02A303105B1F477FF13C06DE2F2
:105870000E94E82A8C0144275527BA014C195D097A
:105880006E097F09CE012AE00E944A2B9C01200F5D
:10589000311F04C02AE00E944A2B9C01C901DF91FC
:1058A000CF911F910F91FF90EF90DF90CF900895CF
:1058B000EF92FF920F931F937B019A010027F7FC51
:1058C0000095102FB801A7010E941C2C1F910F9169
:1058D000FF90EF900895EF92FF920F931F937C013A
:1058E0000E94582C8C01C7010E94F02A9C01200FB5
:1058F000311FC9011F910F91FF90EF9008950E94F1
:105900002E2B0895EF92FF920F931F937C010E941C
:105910007F2C8C01C7010E94F02A9C01200F311FAF
:10592000C9011F910F91FF90EF90089508951F9264
:105930000F920FB60F9211242F933F934F938F9393
:105940009F93EF93FF938091C00082FD1DC0409113
:10595000C60020913706309138062F5F3F4F2F73D6
:1059600030708091390690913A062817390771F006
:10597000E0913706F0913806E950FA4F40833093B2
:1059800038062093370602C08091C600FF91EF9140
:105990009F918F914F913F912F910F900FBE0F903C
:1059A0001F9018951F920F920FB60F9211242F93EC
:1059B0003F938F939F93EF93FF9320917B063091BA
:1059C0007C0680917D0690917E062817390731F478
:1059D0008091C1008F7D8093C10014C0E0917D064D
:1059E000F0917E06E55CF94F208180917D069091D3
:1059F0007E0601968F73907090937E0680937D064D
:105A00002093C600FF91EF919F918F913F912F912D
:105A10000F900FBE0F901F9018958F929F92AF928C
:105A2000BF92CF92DF92EF92FF920F931F93DF937B
:105A3000CF93CDB7DEB7FC011382128288EE93E0DC
:105A4000A0E0B0E084839583A683B7838DEE93E0D6
:105A5000918380837587648757874687318B208B36
:105A6000138B028BF58AE48AD78AC68AB18EA08E00
:105A7000938E828E8F85848F8889858F8989868F82
:105A80008A89878F8B8980A3CF91DF911F910F9196
:105A9000FF90EF90DF90CF90BF90AF909F908F904E
:105AA0000895AF92BF92DF92EF92FF920F931F93F0
:105AB000CF93DF93EC017A018B01DD24403081EE3E
:105AC000580780E0680780E0780711F0DD24D39460
:105AD00091E0A92EB12CEC89FD89DD2069F0C5018A
:105AE00008A002C0880F991F0A94E2F7808360E043
:105AF00079E08DE390E005C0108260E874E88EE103
:105B000090E0A80197010E94112F215030404040A1
:105B10005040569547953795279580E120303807B6
:105B200020F0DD2011F0DD24D6CFE889F98930831B
:105B3000EA89FB89208319A2EE89FF89408121E04F
:105B400030E0C9010C8C02C0880F991F0A94E2F75B
:105B5000482B4083EE89FF894081C9010D8C02C02A
:105B6000880F991F0A94E2F7482B4083EE89FF893A
:105B70004081C9010E8C02C0880F991F0A94E2F778
:105B8000482B4083EE89FF8980810F8C02C0220F51
:105B9000331F0A94E2F7209528232083DF91CF91C9
:105BA0001F910F91FF90EF90DF90BF90AF900895FD
:105BB000DC011C96ED91FC911D97E05CFF4F21915B
:105BC000319180819181281B390B2F733070C9016D
:105BD00008958FE796E00E94D82D892B11F00E943E
:105BE000962C0895DC011C96ED91FC911D97E05CCC
:105BF000FF4F20813181E054F040DF01AE5BBF4FA9
:105C00008D919C9111972817390719F42FEF3FEFC9
:105C100007C08D919C91E80FF91F8081282F30E0FB
:105C2000C9010895DC011C96ED91FC911D97E05C83
:105C3000FF4F20813181E054F040DF01AE5BBF4F68
:105C40008D919C9111972817390719F42FEF3FEF89
:105C500010C08D919C911197E80FF91F20818D91B3
:105C60009C91119701968F73907011969C938E93CF
:105C700030E0C9010895DC0191968C9191978823B9
:105C800039F05496ED91FC915597808186FFF9CFBC
:105C900091961C920895CF93DF93EC01EE85FF85DA
:105CA000E05CFF4F20813181E054F0402F5F3F4F97
:105CB0002F733070DF01AE5BBF4F8D919C911197B8
:105CC00028173907D1F3E05CFF4F80819181E054C0
:105CD000F040E80FF91F6083EE85FF85E05CFF4F21
:105CE00031832083EE89FF89208181E090E00F8C51
:105CF00002C0880F991F0A94E2F7282B208381E0C5
:105D000089A3EC89FD8980818064808381E090E0B3
:105D1000DF91CF9108958F929F92AF92BF92CF92D1
:105D2000DF92EF92FF920F931F9300D000D00F925B
:105D3000EDB7FEB7319684E0ADB7BEB711968C9340
:105D400083E0818387E0828385E0838381E08483AD
:105D50008FE796E067EF75E04BE356E025EC30E027
:105D600004EC10E0B0ECEB2EF12CA1ECCA2ED12CFF
:105D7000F2ECAF2EB12CE6EC8E2E912C0E940D2D64
:105D80000F900F900F900F900F901F910F91FF9019
:105D9000EF90DF90CF90BF90AF909F908F9008953D
:105DA000CF93DF930E9491290E945827C9EEDDE22C
:105DB0000E94F2132097E1F30E94E92DF9CF629F30
:105DC000D001739FF001829FE00DF11D649FE00DF3
:105DD000F11D929FF00D839FF00D749FF00D659F54
:105DE000F00D9927729FB00DE11DF91F639FB00D53
:105DF000E11DF91FBD01CF011124089597FB092E64
:105E000007260AD077FD04D049D006D000201AF426
:105E1000709561957F4F0895F6F7909581959F4F06
:105E20000895A1E21A2EAA1BBB1BFD010DC0AA1FDB
:105E3000BB1FEE1FFF1FA217B307E407F50720F0F3
:105E4000A21BB30BE40BF50B661F771F881F991F6E
:105E50001A9469F760957095809590959B01AC01B7
:105E6000BD01CF01089597FB092E05260ED057FDE1
:105E700004D0D7DF0AD0001C38F4509540953095F7
:105E800021953F4F4F4F5F4F0895F6F790958095BE
:105E9000709561957F4F8F4F9F4F0895AA1BBB1B35
:105EA00051E107C0AA1FBB1FA617B70710F0A61B1A
:105EB000B70B881F991F5A95A9F780959095BC013B
:105EC000CD010895EE0FFF1F0590F491E02D099488
:105ED000911106C0803219F089508550D0F708958D
:105EE0009927882708952F923F924F925F926F9241
:105EF0007F928F929F92AF92BF92CF92DF92EF925A
:105F0000FF920F931F93CF93DF93CDB7DEB7CA1BDA
:105F1000DB0B0FB6F894DEBF0FBECDBF09942A8805
:105F2000398848885F846E847D848C849B84AA84AD
:105F3000B984C884DF80EE80FD800C811B81AA813A
:105F4000B981CE0FD11D0FB6F894DEBF0FBECDBF05
:085F5000ED010895F894FFCF64
:105F58004E6F005965730054582074696D656F75EC
:105F68007421006D6F64756C65206C6F636B65647C
:105F78003F00486F70206368616E6E656C2000207A
:105F880040200053004E2F4100386368002C002C3D
:105F9800205B005D20280029004E4F5420454E41CB
:105FA800424C45440053656E64696E67207365749E
:105FB80074696E677320746F2052580A00526573B3
:105FC800657474696E672073657474696E6773208D
:105FD8006F6E2052580A0041626F727465642065C2
:105FE800646974730A00696E76616C69642073650C
:105FF8006C656374696F6E000D0A496E76616C6931
:106008006420696E707574202D20646973636172F1
:106018006465642107007363616E6E6572206D6F3D
:1060280064650053657474696E677320736176657F
:106038006420746F20454550524F4D0A00526576D2
:1060480065727465642073657474696E677320661D
:10605800726F6D20454550524F4D0A004C6F616478
:10606800656420666163746F727920646566617522
:106078006C74730A004B657920616E6420636861F3
:106088006E6E656C732072616E646F6D697A65649B
:106098000A004E65772070726F66696C653A004C2D
:1060A8006F616465642073657474696E67732066D4
:1060B800726F6D20454550524F4D0A00454550526C
:1060C8004F4D2064617461206E6F742076616C6935
:1060D800642C207265696E6974696E670A00456E82
:1060E800746572696E672062696E64696E67206D97
:1060F8006F64650A004F70656E4C52536E6720548A
:1061080058207374617274696E672000206F6E2066
:106118004857200050504D005253534900534441B2
:106128000053434C00525844005458440041494ECF
:10613800004C424545500053504B54524D00534279
:1061480055530053554D44004C4C494E44000034BF
:106158002B34003800382B340031320031322B34E4
:106168000031360001000000C01200001A400AA1E8
:10617800204EA5001B1E27522C2330802500000529
:10618800400AA1204EA50020244EA52C2330004B08
:10619800000006400AD0009D49007B289D492C2319
:1061A8003000E1000005400A4501D7DC03B81E0EA7
:1061B800BF00232E48E801008A400A6001555502B5
:1061C800AD1E20000023C88025000005400AA1203C
:1061D8004EA50020244EA52C233000020002000208
:1061E8000002000200020002000200020002000297
:1061F80000020002000200020002FFC402C802CD31
:1062080002D102D502D902DD02E102E702EE02F371
:1062180002F802FE02FE02FE02FE023501FF020340
:1062280003050309030C031103350100070B0C10C8
:10623800111500160A13223129000000004B2E9B6D
:0A6248002AD82D122EF22D3B2E0055
:00000001FF
